:020000020000FC
:10000000A3C947C20000000025C000004DC1000088
:10001000000050C1000000000000000002030406C0
:10002000080C101820304060800002030406080C01
:10003000101820304080FF000406080C10182030F3
:10004000406080A0C0000D0D0405060D050D0602E0
:10005000030302004FB662FD1EC070FF18C165FDAC
:10006000F8C00994C0919700C395C0939700C5E06C
:10007000C519B8F3D0919700CD1B98F3C8E7089441
:1000800083FDC795C4BDC52DCC2321F4C0E083FDFD
:10009000C0E8C4BD07C171FF03C0919890989398C0
:1000A000C52D089483FDC795C4BDC09399006B7F8F
:1000B000C52DCF3F09F441C0C0919800C395C093AE
:1000C000980070FF35C09198909893984FBE1895FE
:1000D0007860C091A000CC2391F0C0919800CA959F
:1000E000D091A000CD1B58F0777FC0919800D0919F
:1000F0009F00CD1B08F41CC02092980019C0919855
:1001000090989398C5E0CA95F1F7C0917500CA958B
:10011000C2FD09C0C1FD05C095FF959A95FD949A51
:100120000EC0979A0CC095FF949A95FD959A07C0BA
:100130009198909893984FBE1895209299004FBE31
:100140001895A5C0552021F095FF919A95FD939A99
:1001500090989DC0552009F0909A95FF939895FD31
:10016000919895C0552021F095FF939A95FD919A0D
:1001700095FF919895FD93988AC095FF949895FD69
:10018000959895FF959895FD9498C5E0CA95F1F7D7
:10019000552021F095FF919A95FD939A909877C0FC
:1001A00095FF949895FD95989798C5E0CA95F1F7B5
:1001B000552021F095FF919A95FD939A909867C0EC
:1001C000979895FF949895FD9598C5E0CA95F1F795
:1001D000552009F0909A95FF939895FD919857C0F6
:1001E000979895FF959895FD9498C5E0CA95F1F775
:1001F000552009F0909A95FF939895FD919847C0E6
:1002000095FF959895FD94989798C5E0CA95F1F754
:10021000552021F095FF939A95FD919A95FF91981D
:1002200095FD939834C095FF959895FD949895FF0A
:10023000949895FD9598C5E0CA95F1F7552021F061
:1002400095FF939A95FD919A95FF919895FD9398B6
:100250001EC082FF1CC0C0917500C2FD0BC0C1FD55
:1002600011C095FF949895FD959895FF959895FDEB
:1002700094980DC0C1FDF5CF95FF949895FD959884
:10028000979805C0979895FF959895FD9498C52DDA
:10029000C095089483FDC795C4BDC0939900209272
:1002A000970064604FBE18954FB6C0E1C8BF6E7F1F
:1002B0004FBE18953FB68F7EABB7A074A211806178
:1002C000A0E0ABBFA9B7AE7FA9BF7894A0916600AC
:1002D000AA2349F0A92FAF7151F1A0916600AA9508
:1002E000A093660024C040E050E0A0B396FFA09524
:1002F000A2FD4FEF96FDA3E096FFA2E0A5BFAA27BF
:10030000A064AABF8D7FA0B396FFA095A2FD5FEF6A
:10031000451749F7A8E161FDA0936600A92FAF71C9
:1003200019F0A8E1A093660040938D008160A09130
:100330006700AA2331F0A0916700AA95A0936700F7
:1003400007C0A92FAF7121F08061AA27A064AABFBE
:1003500080FF4BC0A0918D004A2F8E7FA92FAF71D7
:10036000E1F0A091AE00A430C1F4403F08F040EFAE
:10037000A42FA295AF704A0F5091B000533069F08E
:10038000A695A69550FD01C0A69552FD03C0A41BDD
:100390004A2F03C04A0F08F44FEF4093610071FFEA
:1003A00008C0A091610050919200A51710F05093E1
:1003B00061004091AE00443029F5A0916100409168
:1003C0006300A41B70F04091CF00A40B50F0A091EB
:1003D0006300A40FA093630040F4AFEFA093630009
:1003E00004C0A0916100A093630040916300A091BC
:1003F00092004A1708F04A2FA09194004A1708F07B
:100400004A2F542EA52DA03408F06860A0916000FA
:10041000A395A093600051F0F894A9B7A160A9BF7B
:1004200084FF02C0A0E4ABBF3FBE189541E05091ED
:100430006600552331F0A92FAF7119F45A955093E6
:100440006600A0918D00A13018F0209290000DC0A0
:100450002092910020929A00A0919000AF5FA0930B
:10046000900018F0AFEFA0939000A0919300A65FCA
:1004700020F05FEF5093930002C0A0939300F89494
:10048000A9B7A160A9BF84FF02C0A0E4ABBF3FBE73
:1004900018953FB64CB55DB58F7EABB7A074A21171
:1004A0008061A0E0ABBFA9B7AE7FA9BF789481FD02
:1004B00026C096FDA2E096FFA3E0A5BF8260A0B390
:1004C00096FFA095A2FF05C040936400509365007D
:1004D00033C196FDA3E096FFA2E0A5BFAA27A064C2
:1004E000AABF8D7FA92FAF7109F417C140E0A0B357
:1004F00096FFA095A2FD11C140938D0004C196FD09
:10050000A3E096FFA2E0A5BF8D7F61FF6BC096FDC3
:10051000A2E096FFA3E0A5BFAA27A064AABF8260BD
:100520004093880050938900A09086004A19B090AB
:1005300087005B09BB24A2E0EA2EA22C483CA0E085
:100540005A0730F4A0E1BA2EE22CAAE0AA2E27C066
:100550004836A1E05A0730F4A8E0BA2EE22CAFE00A
:10056000AA2E1DC0403DA2E05A0730F4A4E0BA2EE6
:10057000E22CAEE1AA2E13C0403AA5E05A0730F4AF
:10058000A2E0BA2EE22CACE3AA2E09C04839A8E0BA
:100590005A0728F4A1E0BA2EE22CA8E7AA2EC42E0E
:1005A000A0918A00CA1AD52EA0918B00DA0ADD200C
:1005B0002AF4AFEFC094D094CA1ADA0A20928C00C1
:1005C000CA14DE0418F4A1E0A0938C0040938A00C2
:1005D00050938B0040918800509189004093860091
:1005E00050938700A09164004A1BA09165005A0BAC
:1005F00094FD7CC093FD7AC092FD76C056954795D8
:1006000091FD72C05695479590FD6EC0D52EC42EB3
:10061000D694C79461FD0CC0AC2DAC51AD2DA24059
:1006200008F07BC0DD2021F4AC2DA85C08F475C077
:10063000A0E0EA2E97FD08C0E090C200A091B400AF
:10064000A33011F4E090CA00AAEFEA0EF22CF21CDB
:10065000CE18DF084FB74170A091B400A330A9F4C1
:10066000442329F095FD11C0F894906204C095FFD1
:100670000CC0F8949F7D919890989398949897982F
:10068000959871FD01C060687894442369F0A09149
:10069000B400A33031F4AFEFC094D094CA1ADA0A90
:1006A00003C040E050E022C0A091B400A33049F460
:1006B000CC0CDD1CA5E0CA1AD20818F4A0E0CA2EA2
:1006C000D22CAFEFCA16D20418F04FEF50E00EC094
:1006D000F090A700CF9C412D000C441F50E008F083
:1006E00012C04FEF50E00FC05695479594FF07C0DA
:1006F000552309F04FEFA42FA6954A0F521D4F3FE7
:10070000520508F04FEF40938D00816061FF05C0F6
:10071000AFE1A095A923AB299A2FA8E1A093660089
:10072000A92FAF7119F4AAE0A093660061FD04C07F
:10073000A92FAF7109F08F7EA6E0A0936700A92FC3
:10074000AF7119F4AAE0A0936700F894A9B7A1606B
:10075000A9BF84FF02C0A0E4ABBF3FBE189511E063
:100760000AC013E008C01AE006C01EE104C014E687
:1007700002C018EC00C005E1BB27BA95F1F70A9555
:10078000D9F71A95C1F708952AE338E709C020E39D
:100790003CE806C02AE234EB03C025E238EC00C096
:1007A000652CB1E05B2E12E095FD9F7D95FF906278
:1007B000BB279798BA95F1F7552009F0909ABA950A
:1007C000F1F79098BA95F1F7979ABA95F1F7552005
:1007D00021F095FF919A95FD939AB091A800BA9552
:1007E000F1F795FF919895FD9398B7E8BA95F1F7D1
:1007F0001A95D1F6022FB22FBA95F1F70A95D9F7CB
:100800003A9571F69798562C0895221B39E0001FEF
:100810003A9509F40895221F211B18F4210F88949A
:10082000F6CF0894F4CF622C722CB0E08894B39584
:10083000221F331FE0F7379527958894912E802E3D
:10084000020B130B10F4192D082D10F4889401C01D
:100850000894661C771CBA9571F7172D062D08951C
:10086000322D11232AF43A9500951095031B130B92
:10087000F894029F712C002D129F912C802C78945B
:10088000780C172D921C292DB4E06B2E2695179508
:1008900007956A94D9F7332321F000951095031B2F
:1008A000130B08950091AE000430A1F1B0918D00BA
:1008B000B15008F010C0B0916100B0936300209275
:1008C0007700209278002092790020927A0020927E
:1008D0007B006F7B1FC06090AE006064B0916100D0
:1008E000B093620008E317EC20917300309174001C
:1008F00036952795B62DBA9541F036952795B62DA4
:10090000BA95BA9511F0369527958DDF009377004B
:1009100010937800089566FF1BC000917700B09196
:1009200062000B1B10917800120928F40038BFEF09
:100930001B0740F009C00F37120508F405C00FE788
:1009400010E002C000E81FEF00937C0010937D00D0
:10095000089566FF39C000917C00B09179000B0FBB
:1009600010917D00B0917A001B1F20E030917D0036
:1009700033230AF42A95B0917B002B1F1AF4203FF1
:1009800040F00AC02F3008F407C00FEF1FEF2FE030
:1009900003C000E010E020EF30916300B0919200BE
:1009A0003B1718F4332331F009C0B0917D00BB230D
:1009B0005AF004C0B0917D00BB2332F4009379005B
:1009C00010937A0020937B00089566FF2FC020913A
:1009D000CD0000917C00000F10917D00111F40DFC1
:1009E00011232AF40038BFEF1B0740F009C00F376E
:1009F000120508F405C00FE710E002C000E81FEF81
:100A0000002352F0B0916200B01B0B2F18F00130A0
:100A100008F00AC001E008C000950F5FB0916200C5
:100A20000B0F08F001C00FEF00937E00089566FFE2
:100A30002DC02091CE0000917A0010917B0010DF34
:100A400011232AF40130BFEF1B0740F009C00F3F0C
:100A5000120508F405C00FEF10E002C001E01FEF1F
:100A6000112352F0B0917E00B01B0B2F18F0013013
:100A700008F00AC000E008C000950F5FB0917E004A
:100A80000B0F08F001C00FEF0093630008950FEF04
:100A9000677FB72FB670E9F46860B0917400B83022
:100AA00008F0677FB0917400A1F00FEF109174000F
:100AB000ACDEF894B09170000B9F112D002D78944E
:100AC000112309F00FEFB09195000B1710F400916E
:100AD00095000093940008951ED374FFB7E074FD51
:100AE000B7E0B068B064B7B9B6B1B068B064B6B9D1
:100AF00036DE74FFB7E074FDB7E0B068B064B7B934
:100B0000B6B1B068B064B6B9B6B1B6FDFDCF04B148
:100B100015B1B6B1BF77B6B943D32DE62093A30084
:100B200030E03093A400732E7694622E6694620EA9
:100B3000731E262D372D0217130778F08090A3001F
:100B4000BDE6B80DB093A3008090A400B0E0B81D3E
:100B5000B093A400260D371DEECF8090A300909097
:100B6000A4001091A40016950091A3000795169576
:100B70000795B091A300B00FB093A100B091A4006D
:100B8000B11FB093A20023E0169507952A95E1F7CF
:100B90002091AF002A9529F42092A3002092A4006E
:100BA0000AC02A9521F0800E911E2A95E1F78092C5
:100BB000A3009092A40008952091AF00B6B1B6FDB5
:100BC000FBCF04B115B1B6B1BF77B6B9B091A500EE
:100BD000B395B093A500B83060F12092A500B09114
:100BE000CC00BB2321F1112329F0B091A600BF3F17
:100BF00061F009C0B091A6000B1739F020F4BB23B7
:100C000021F0BA9502C0B395E1F300919200B09340
:100C1000A600B03050F400ECB03038F400E8B0304A
:100C200020F400E4B03008F400E0009392007F7EEE
:100C30000895213099F00F3FB3E01B0778F4B0918D
:100C4000A3000B17B091A4001B0740F4B0919200D1
:100C5000BB23A9F0BA95B093920011C0B091920055
:100C6000BF3F69F0B395B0939200B091B400B33038
:100C700031F4B0919200BC5F10F4B09392000091F7
:100C80009200B0916300B01B10F400916300B0912A
:100C900093000B1750F000919300B0919300BF3F69
:100CA00021F0B0919300B0939200B091AE00B430B7
:100CB00009F406C0B09194000B1708F00B2F502ECA
:100CC000B091A500B73009F47061089502E3F8947B
:100CD000B091D0000B9F012D000C001F7894B091B3
:100CE00092000B1710F000919200009361000093A6
:100CF0006300502E00939500089520927300B8E091
:100D0000B093740008952091800030918100F89490
:100D10000CB51DB5200F311F3BBD2ABD6160B0E190
:100D2000B8BF7894209171003091720000937100E7
:100D300010937200021B130B20917300309174000A
:100D4000622E732EB4E08B2EB2E09B2EB091740015
:100D5000B43010F08A949A94B83010F08A949A942F
:100D6000769467948A94E1F726193709992021F03F
:100D7000169507959A94E1F7200F311F2093730081
:100D80003093740008F00895BFEFB0937300B093F0
:100D9000740008952091820030918300F8940CB57E
:100DA0001DB5020F131F1BBD0ABD6160B0E1B8BFC6
:100DB0007894089560FDFECFEDDF0895B091BE00F8
:100DC00000916E00023808F0B395003A08F0B39530
:100DD000B63008F0B5E09B2EBCE08B2EB0917400CD
:100DE000B33030F48394839482FF02C0839483945D
:100DF000B23030F48394839482FF02C0839483944E
:100E000071FF03C0B3E09B2E822C109174000091FF
:100E1000730024E0169507952A95E1F70819120941
:100E200028F0B02FB250B12FB20910F402E010E058
:100E3000312F202F712E602E76946794B92DB33008
:100E4000E9F0B0FD05C0060D171D262D372D06C093
:100E5000000F111F0250120922E030E0B92DB3300B
:100E600068F02093840030938500009380001093F5
:100E70008100609282007092830008950093840044
:100E8000109385002093800030938100609282004F
:100E900070928300089560FDFECF20918200220FA2
:100EA00030918300331FB72FB67021F0209173006B
:100EB00030917400F8940CB51DB5020F131F1BBDC3
:100EC0000ABD6160B0E1B8BF789408956061209276
:100ED000760020E004C060612092760020E2B72F07
:100EE000B67009F06F7E789460FD05C0B091760011
:100EF000BB2309F0089501E063FF0AC0B0917400BC
:100F0000B33008F002E0B0917400B63008F003E0AE
:100F100071FF01C006E060FD06C0B0917600BB2302
:100F200011F0789408951AE083FF1AE07894000095
:100F30000000F89462FD03C014E183FF14E171FF27
:100F400001C018E7B4B530919900B31BB10B18F389
:100F5000B0917600B395B0937600B5E03B2F6B2E41
:100F6000722CB8B1B072B21709F073943A95C9F700
:100F70007394761488F464FFB2CF6F7E3CB56DB481
:100F80007090730080907400370D681C6BBC3ABD84
:100F90006160B0E1B8BFA3CF64FDA1CF0A9509F0AD
:100FA000BACF7894089571FF0AC0B0916D00B395DF
:100FB000B0936D0060FD0CC020926D0009C060FD13
:100FC00007C064FD05C067FD03C0BF91BF9169C440
:100FD00008952091840030918500F8940CB51DB5DA
:100FE000020F131F1BBD0ABD6160B0E1B8BF78944A
:100FF0000895EFDF00E063FF03C064FF01C001E07C
:10100000F89410916E00B7E01B9F212D102D78945D
:10101000200F2695179526951795269517951093C9
:101020006E00183718F4B8E7B0936E0000916E00A8
:10103000B0916F000B1720F0606291989098939890
:1010400060FDFECF0895F89494989798959882FF44
:1010500007C0E0E0F1E073FF03C0BEE1BA95F1F72D
:1010600095FF949A95FD959AB2E0B093750089C06A
:10107000F89495FF939895FD919882FF0DC0E0EF4D
:10108000F0E073FF0BC0979895FF959895FD9498A5
:10109000BEE1BA95F1F702C0EAEAF0E062FF03C0F0
:1010A000552009F0909AB3E0B09375006AC0F894A7
:1010B00094989798959882FF07C0E0EEF0E073FF50
:1010C00003C0BEE1BA95F1F795FF959A95FD949A04
:1010D000B4E0B093750055C0F894909882FF0DC0AD
:1010E000E0EDF0E073FF0BC095FF949895FD9598A7
:1010F0009798BEE1BA95F1F702C0E2EAF0E062FF2C
:1011000006C0552021F095FF919A95FD939AB5E080
:10111000B093750036C0F89494989798959882FF8C
:1011200007C0EDEBF0E073FF03C0BEE1BA95F1F745
:10113000979AB6E0B093750024C0F89495FF919803
:1011400095FD939882FF10C0E3E1F1E073FF0EC0BC
:1011500095FF949895FD959895FF959895FD949891
:10116000BEE1BA95F1F702C0E2EBF0E062FF06C023
:10117000552021F095FF939A95FD919AB1E0B09397
:10118000750067FF0AC00CD0BEE1BA95F1F7B5E073
:10119000BA95F1F7949A979A959A6F7D78940895F5
:1011A00021EA30E0F9019198909893989498979853
:1011B00095986B7F0895ACEAB0E009E00D9309E0E3
:1011C0000D9304E00D9301E00D9303E00D930FEFF9
:1011D0000D930AE00D9301E00D9301E00D9301E002
:1011E0000D93A8EBB0E001E00D930FEF0D930D937D
:1011F0000FEF0D930D930D9303E00D9306E00D9308
:101200000FEF0D930D9305E20D9300ED0D9308E2A2
:101210000D9300E50D9304E00D930DE00D9302E0B6
:101220000D9300E00D930AE70D930FEF0D9301E08E
:101230000D9308952091BF0009E011E0223011F4D0
:1012400005E011E0233011F405E012E0243011F440
:1012500005E013E0253011F409E017E0263011F421
:1012600000E010E000939F001093A0002091B300D5
:101270008B7F777FB091B400B33019F09F7DB1FDC3
:1012800090629F7BB091B500B1FD9064B22FB230F7
:1012900011F0886001C0877F0895ECE1F0E00091D3
:1012A000AC000A95E00FF21DB491B093CD0000910F
:1012B000AD000A95E00FF21DB491B093CE0070DF3F
:1012C0000895EAE2F0E00091C7000A95E00FF21DF0
:1012D000B491B093CF0064DF0895E8E3F0E00091AB
:1012E000B2000A95E00FF21DB491B093D00058DF20
:1012F00008950895B091C8000FEF1CE0B23011F4CA
:1013000000EA1AE0B33011F402E815E000936F0030
:1013100010937000089508952091C2003091C30089
:1013200097FF02C020E03FEFB32FB21B6B2EB258E5
:1013300010F4B2E86B2E00E00395609EB12DB0581A
:10134000D8F30093A7000895F894E3E0F0E0B9E043
:10135000B7BFB491B078C1F3F894A895B1B5B861AE
:10136000B1BDB0E0B1BDB4E0BEBFBFE5BDBF18DFE9
:10137000B0E0B8BBB0E1B7BBB0E0B5BBB0E0B4BB68
:10138000B0E0B2BBBBEBB1BB2224A0E0B0E02D9239
:10139000AA31E9F7A0E6B0E00FEF2D920A95E9F740
:1013A0000ADF9FD247DF79DF8CDF97DFA2DFA2DF82
:1013B000B2DFB2DF0091C4000093A800F1DEB2E01A
:1013C000B3BFB2E0BEBDB2E0B5BDF894D2D9DCD9AE
:1013D000CCD9DDD9CAD9DED9C8D9CBD9CAD9C7D9D0
:1013E000B1E5B8BFB9BFB0B7B860B0BFB6B1B4600F
:1013F000B6B9B5D9789470DBB0E4BBBFBB27B06495
:10140000BABF8D7FB6D9B1E0B0936900626025E0C4
:10141000B0918C00BB2309F425E0A3D9B0918D00D5
:10142000B230A8F3B92FBF7100918F0000938E00E6
:10143000B0938F00B01759F72A9551F76D7F96FD3D
:10144000B3E096FFB2E0B5BFBB27B064BABF8D7FF3
:101450008ED987D902E0B92FBF7109F400E0B091AD
:101460008D00B017B0F3F8948FD98ED98DD97894B8
:1014700080D920927F00B091B400B33009F472C0DB
:1014800070D9B091B800B13008F46CC0B091690067
:10149000B13008F467C0B92FBF71C1F0B0918D00B1
:1014A000BF3F08F45FC0F89478D9789460D9B091C0
:1014B0008D00B130C0F7F89467D955D965D97894C3
:1014C00056D9B0918D00BF3FB0F3D4C2B3E09B2E8C
:1014D0009068F89421DF78944AD9F8949F771CDFBC
:1014E00080908D00B0918D00BF37789408F442C091
:1014F00036D9F89452D978949A9451F7B82DB550BA
:10150000B093C30036D9F89419D287D27894BAE050
:101510009B2E9068F89400DF789429D9F8949F77EF
:10152000FBDE80908D00B0918D00BF37789478F706
:1015300016D9F89429D917D927D978949A9449F7C4
:10154000B82DBB5FB093C20014D9F894F7D174D210
:1015500078940DD9F894E0DE7894B0918D00BF3F77
:10156000C0F388C200918D00B0917F000B1710F07E
:1015700000937F00FCD801E0B091B400B35009F4AF
:1015800005E0B0918D00B01708F075CFF89405D93B
:1015900004D903D97894EDD82092690020926A008A
:1015A00020926B00B0916A00B395B0936A00BF3F80
:1015B00069F5B0916B00B395B0936B00B091C60024
:1015C00009E1BA9559F002E3BA9541F00DE7BA95F1
:1015D00029F00AEFBA9511F020926B00B0916B00E0
:1015E000B017A0F0B0916B00BA95B0936B00B4EB5C
:1015F000B0936A00B091C500B093A800F894CDD81C
:101600007894B091C400B093A800B1D8ACD8B09190
:101610006600BB2321F4B92FBF7109F4F7CEB09156
:101620008D00B63008F4BECFB091B400B35009F0CD
:101630009ED8B0916600BB2309F4E8CEF894B0DDE3
:10164000209261002092620020926300522C7894D4
:10165000B091B100B093960020927700209278006C
:101660002092790020927A0020927B002092A5009F
:1016700060E070E020926E0040DBB8E0B093A5001F
:1016800070616DD874FFB7E074FDB7E0B068B06406
:10169000B7B9B6B1B068B064B6B9B6B1B6FDFDCFF2
:1016A00004B115B1B6B1BF77B6B9112309F00FEF88
:1016B0000093A60081DAB8E0B093A5007061809035
:1016C000B300B2E0B093B300B5DD8092B300F894FC
:1016D000BFEFB0939200FADAB0916100B09392003C
:1016E000B0939300B09394007894B1E0B09361000C
:1016F000B09363005B2EB0939B00B0919100B093C8
:101700009A007160726020926D0005DD16DDFBDAD3
:10171000F4DA54DB04C08EDD2092A5007F7E95FFB5
:10172000B2E095FDB4E0B068B064B7B9D4DB3BDC9F
:1017300050DCB8D85EDC87DCE6DA3CDB3FDBABDBD9
:10174000B3E0B068B064B7B9C1DB2DDC42DCE3D8EC
:101750009ED94FDC8DDCD7DA2DDB30DB9CDB95FFAF
:10176000B4E095FDB2E0B068B064B7B9B4DB1BDC9F
:1017700030DCEFD83EDC9BDCC6DA1CDB1FDB8BDB0E
:1017800095FFB2E095FDB4E0B068B064B7B99EDBF8
:101790000ADC1FDC1AD92DDC9FDCB5DA0BDB0EDB93
:1017A0007ADBB3E0B068B064B7B995DBFCDB11DC81
:1017B0003ED91FDCB0DCA7DAFDDA00DB6CDB95FF7D
:1017C000B4E095FDB2E0B068B064B7B97FDB74FFF8
:1017D000B7E074FDB7E0B068B064B7B9B6B1B0684F
:1017E000B064B6B9E0DBF5DB04DCA7DC8CDAE2DA66
:1017F000E5DAE2D950DB71FF2EC067FD2CC0B09155
:101800009500B0939200B0939300B0919100B09383
:101810009A00B1E0B0939B0014E624E1B0916D0012
:10182000B11798F07D7F746020936C00B091B40084
:10183000B33051F4B0919500B0939200BFEFB093E4
:101840009300B0E2B093940006C0B0918D00B13027
:1018500008F065CF26C072FF10C067FD0EC0B091C2
:101860006C00BA9511F47B7F56CFB0936C00B091A9
:101870008D00B13008F053CF14C0B0919000BA3F42
:1018800080F4B92FBF7121F4B0916600BB2349F0F9
:10189000B091740000EF67FF01C000E6B01708F4D4
:1018A0003ECFF8947DDC8090B300B2E0B093B300FB
:1018B000C1DC8092B30020926100209262002092ED
:1018C0006300522C209296007E7F789448D768DC83
:1018D000B92FBF7129F4B0916600BB2309F496CDEE
:1018E0005DCEEDE0F0E023D0053509F01BC0EEE061
:1018F000F0E01DD00A3A09F015C03AE0ACEAB0E0D9
:10190000E3E0F0E014D00D9331963A95D9F735E144
:10191000A8EBB0E0EFE0F0E00AD00D9331963A95F5
:10192000D9F702C048DC0AD0E4E2F0E00895E1997A
:10193000FECFEEBBFFBBE09A0DB308951ED03AE098
:10194000ACEAB0E0E3E0F0E00D910FD031963A95CB
:10195000D9F735E1A8EBB0E0EFE0F0E00D9105D06C
:1019600031963A95D9F712D00895E199FECF0DBB83
:10197000EEBBFFBBE29AE19A0895EDE0F0E00FEFD5
:10198000F4DFEEE0F0E00FEFF0DF0895EDE0F0E0DF
:1019900005E5EBDFEEE0F0E00AEAE7DF08953091DD
:1019A000A9000091AA00313011F40093AC0032304C
:1019B00011F40093AD00333011F40093AE003430D5
:1019C00011F40093B000353011F40093AF003630BD
:1019D00011F40093B200373011F40093BE00383098
:1019E00011F40093C700393011F40093BF003A306E
:1019F00011F40093B3003B3011F40093C8003C3065
:101A000011F40093B4003D3011F40093B500089533
:101A100025E0AFD62A95E9F70895B6D6B8D6BAD656
:101A2000BCD6A1D6B1D6B3D6B5D6B7D69CD6ACD691
:101A3000AED6B0D6B2D60895B0D6ACD6A8D6A4D677
:101A400092D6ABD6A7D6A3D69FD68DD6A6D6A2D6EB
:101A50009ED69AD608958090A9009090AA0094D618
:101A600093D692D680D68A94D1F797D67CD69A947C
:101A7000E1F70895F894D1DF7894CADFC9DFB1E0C7
:101A8000B093A900B1E0B093AA002092AB00F89403
:101A9000E2DF7894B5E06B2E70908D006AD6B0913D
:101AA0008D007B16C9F7B13018F0BF3F40F107C079
:101AB00076DFF89443DFB1DFB8E0B1BDA9DF6A9407
:101AC00059F7B091AB00B395B093AB00B33008F4C5
:101AD000DECF9EDFB091AA00B395B093AA00F89430
:101AE000B091A900BA95E6E4F0E0EB0FF21D049185
:101AF00078940395B091AA00B01708F4C6CF88DF98
:101B000087DFB091A900B395B093A900B091A90067
:101B1000BE3008F4B7CF4FDBF89410DFB8E0B1BDAA
:021B200077DF6D
:00000001FF
